Microchip MPLAB XC8 Compiler V2.36

Linker command line:

-W-3 --edf=/opt/microchip/xc8/v2.36/pic/dat/en_msgs.txt -cn \
  -h+dist/default/production/lab1Hector.X.production.sym \
  --cmf=dist/default/production/lab1Hector.X.production.cmf -z -Q18F452 \
  -o/tmp/xcXdDomdj --defsym=__MPLAB_BUILD=1 \
  -Mdist/default/production/lab1Hector.X.production.map \
  --md=/tmp/xcXbinadc.dat -E1 -ver=XC8 Compiler --acfsm=1493 \
  -ACODE=00h-03FFFhx2 -ACONST=00h-07FFFh -ASMALLCONST=0600h-06FFhx122 \
  -AMEDIUMCONST=0600h-07FFFh -ACOMRAM=01h-07Fh -AABS1=00h-05FFh \
  -ABIGRAM=01h-05FFh -ARAM=080h-0FFh,0100h-01FFhx5 -ABANK0=080h-0FFh \
  -ABANK1=0100h-01FFh -ABANK2=0200h-02FFh -ABANK3=0300h-03FFh \
  -ABANK4=0400h-04FFh -ABANK5=0500h-05FFh -ASFR=0F80h-0FFFh \
  -ABIGSFR=0F80h-0FFFh -ACONFIG=0300000h-030000Dh -AIDLOC=0200000h-0200007h \
  -AEEDATA=0F00000h-0F000FFh -peeprom_data=EEDATA \
  -preset_vec=00h,intcode,intcodelo,powerup,init -pramtop=0600h \
  -psmallconst=SMALLCONST -pmediumconst=MEDIUMCONST -pconst=CONST \
  -AFARRAM=00h-00h \
  -prdata=COMRAM,nvrram=COMRAM,nvbit=COMRAM,rbss=COMRAM,rbit=COMRAM \
  -pfarbss=FARRAM,fardata=FARRAM,nvFARRAM=FARRAM \
  -pintsave_regs=BIGRAM,bigbss=BIGRAM,bigdata=BIGRAM -pbss=RAM \
  -pidata=CODE,irdata=CODE,ibigdata=CODE,ifardata=CODE -prparam=COMRAM \
  /tmp/xcXaGNkjc.o dist/default/production/lab1Hector.X.production.o 

Object code version is 3.11

Machine type is 18F452



                Name                               Link     Load   Length Selector   Space Scale
/tmp/xcXaGNkjc.o
                idloc                            200000   200000        8        0       5
                config                           300000   300000        E        0       4
                text                               39A4     39A4        2     1CD2       0
                init                                  2        2        4        0       0
                reset_vec                             0        0        2        0       0
dist/default/production/lab1Hector.X.production.o
                idloc                            200000   200000        8        0       5
                config                           300000   300000        E        0       4
                text18                             39BA     39BA        C     1CDD       0
                text17                             3A16     3A16       16     1D0B       0
                text16                             3AA8     3AA8       76     1D54       0
                text15                             3A06     3A06       10     1D03       0
                text14                             39C6     39C6        C     1CE3       0
                text13                             39D2     39D2        C     1CE9       0
                text12                             3A2C     3A2C       18     1D16       0
                text11                             39A6     39A6        A     1CD3       0
                text10                             3D44     3D44       F0     1EA2       0
                text9                              3C68     3C68       DC     1E34       0
                text8                              3BB4     3BB4       B4     1DDA       0
                text7                              3A7E     3A7E       2A     1D3F       0
                text6                              3B1E     3B1E       96     1D8F       0
                text5                              3A44     3A44       18     1D22       0
                text4                              3A5C     3A5C       22     1D2E       0
                text3                              39EA     39EA        E     1CF5       0
                text2                              39DE     39DE        C     1CEF       0
                text1                              39B0     39B0        A     1CD8       0
                text0                              3E34     3E34      1CC     1F1A       0
                cstackCOMRAM                          1        1       16        1       1
                bssCOMRAM                            19       19        2        1       1
                cinit                              39F8     39F8        E     1CFC       0
                nvCOMRAM                             17       17        2        1       1

TOTAL           Name                               Link     Load   Length     Space
        CLASS   CODE           
                text                               39A4     39A4        2         0
                init                                  2        2        4         0
                reset_vec                             0        0        2         0
                text18                             39BA     39BA        C         0
                text17                             3A16     3A16       16         0
                text16                             3AA8     3AA8       76         0
                text15                             3A06     3A06       10         0
                text14                             39C6     39C6        C         0
                text13                             39D2     39D2        C         0
                text12                             3A2C     3A2C       18         0
                text11                             39A6     39A6        A         0
                text10                             3D44     3D44       F0         0
                text9                              3C68     3C68       DC         0
                text8                              3BB4     3BB4       B4         0
                text7                              3A7E     3A7E       2A         0
                text6                              3B1E     3B1E       96         0
                text5                              3A44     3A44       18         0
                text4                              3A5C     3A5C       22         0
                text3                              39EA     39EA        E         0
                text2                              39DE     39DE        C         0
                text1                              39B0     39B0        A         0
                text0                              3E34     3E34      1CC         0
                cinit                              39F8     39F8        E         0

        CLASS   CONST          

        CLASS   SMALLCONST     

        CLASS   MEDIUMCONST    

        CLASS   COMRAM         
                cstackCOMRAM                          1        1       16         1
                bssCOMRAM                            19       19        2         1
                nvCOMRAM                             17       17        2         1

        CLASS   ABS1           

        CLASS   BIGRAM         

        CLASS   RAM            

        CLASS   BANK0          

        CLASS   BANK1          

        CLASS   BANK2          

        CLASS   BANK3          

        CLASS   BANK4          

        CLASS   BANK5          

        CLASS   SFR            

        CLASS   BIGSFR         

        CLASS   CONFIG         
                config                           300000   300000        E         4

        CLASS   IDLOC          
                idloc                            200000   200000        8         5

        CLASS   EEDATA         

        CLASS   FARRAM         

        CLASS   HEAP           

        CLASS   STACK          



SEGMENTS        Name                           Load    Length   Top    Selector   Space  Class

                text2                          0039DE  00000C  0039EA      1CEF       0  CODE    
                text3                          0039EA  00000E  0039F8      1CF5       0  CODE    
                reset_vec                      000000  000006  000006         0       0  CODE    
                text13                         0039D2  00000C  0039DE      1CE9       0  CODE    
                cinit                          0039F8  00000E  003A06      1CFC       0  CODE    
                text14                         0039C6  00000C  0039D2      1CE3       0  CODE    
                text18                         0039BA  00000C  0039C6      1CDD       0  CODE    
                text15                         003A06  000010  003A16      1D03       0  CODE    
                text12                         003A2C  000018  003A44      1D16       0  CODE    
                text17                         003A16  000016  003A2C      1D0B       0  CODE    
                text                           0039A4  000002  0039A6      1CD2       0  CODE    
                text11                         0039A6  00000A  0039B0      1CD3       0  CODE    
                text1                          0039B0  00000A  0039BA      1CD8       0  CODE    
                text5                          003A44  000018  003A5C      1D22       0  CODE    
                text0                          003E34  0001CC  004000      1F1A       0  CODE    
                text10                         003D44  0000F0  003E34      1EA2       0  CODE    
                cstackCOMRAM                   000001  00001A  00001B         1       1  COMRAM  
                text16                         003AA8  000076  003B1E      1D54       0  CODE    
                text7                          003A7E  00002A  003AA8      1D3F       0  CODE    
                text4                          003A5C  000022  003A7E      1D2E       0  CODE    
                text9                          003C68  0000DC  003D44      1E34       0  CODE    
                text8                          003BB4  0000B4  003C68      1DDA       0  CODE    
                text6                          003B1E  000096  003BB4      1D8F       0  CODE    


UNUSED ADDRESS RANGES

        Name                Unused          Largest block    Delta
        BANK0            000080-0000FF               80
        BANK1            000100-0001FF              100
        BANK2            000200-0002FF              100
        BANK3            000300-0003FF              100
        BANK4            000400-0004FF              100
        BANK5            000500-0005FF              100
        BIGRAM           00001B-0005FF              5E5
        BIGSFR           000F80-000FFF               80
        CODE             000006-0039A3             399E
                         004000-007FFF             4000
        COMRAM           00001B-00007F               65
        CONST            000006-0039A3             399E
                         004000-007FFF             4000
        EEDATA           F00000-F000FF              100
        MEDIUMCONST      000600-0039A3             33A4
                         004000-007FFF             4000
        RAM              000080-0005FF              100
        SFR              000F80-000FFF               80
        SMALLCONST       000600-0039A3              100
                         004000-007FFF              100

                                  Symbol Table

?___awdiv                                                        cstackCOMRAM 000007
?___awmod                                                        cstackCOMRAM 000001
?___wmul                                                         cstackCOMRAM 000001
_A                                                               nvCOMRAM     000018
_ADCON1                                                          (abs)        000FC1
_B                                                               nvCOMRAM     000017
_LATD                                                            (abs)        000F8C
_LATDbits                                                        (abs)        000F8C
_PORTA                                                           (abs)        000F80
_PORTB                                                           (abs)        000F81
_TRISA                                                           (abs)        000F92
_TRISB                                                           (abs)        000F93
_TRISC                                                           (abs)        000F94
_TRISD                                                           (abs)        000F95
__HRAM                                                           (abs)        000000
__Habs1                                                          abs1         000000
__Hbank0                                                         bank0        000000
__Hbank1                                                         bank1        000000
__Hbank2                                                         bank2        000000
__Hbank3                                                         bank3        000000
__Hbank4                                                         bank4        000000
__Hbank5                                                         bank5        000000
__Hbigbss                                                        bigbss       000000
__Hbigdata                                                       bigdata      000000
__Hbigram                                                        bigram       000000
__Hbigsfr                                                        bigsfr       000000
__Hbss                                                           bss          000000
__HbssCOMRAM                                                     bssCOMRAM    000000
__Hcinit                                                         cinit        000000
__Hclrtext                                                       clrtext      000000
__Hcomram                                                        comram       000000
__Hconfig                                                        config       30000E
__Hconst                                                         const        000000
__HcstackCOMRAM                                                  cstackCOMRAM 000000
__Hdata                                                          data         000000
__Heeprom_data                                                   eeprom_data  000000
__Hfarbss                                                        farbss       000000
__Hfardata                                                       fardata      000000
__Hheap                                                          heap         000000
__Hibigdata                                                      ibigdata     000000
__Hidata                                                         idata        000000
__Hidloc                                                         idloc        200008
__Hifardata                                                      ifardata     000000
__Hinit                                                          init         000006
__Hintcode                                                       intcode      000002
__Hintcode_body                                                  intcode_body 000000
__Hintcodelo                                                     intcodelo    000002
__Hintentry                                                      intentry     000000
__Hintret                                                        intret       000000
__Hintsave_regs                                                  intsave_regs 000000
__Hirdata                                                        irdata       000000
__Hmediumconst                                                   mediumconst  000000
__HnvCOMRAM                                                      nvCOMRAM     000000
__HnvFARRAM                                                      nvFARRAM     000000
__Hnvbit                                                         nvbit        000000
__Hnvrram                                                        nvrram       000000
__Hparam                                                         rparam       000000
__Hpowerup                                                       powerup      000002
__Hram                                                           ram          000000
__Hramtop                                                        ramtop       000600
__Hrbit                                                          rbit         000000
__Hrbss                                                          rbss         000000
__Hrdata                                                         rdata        000000
__Hreset_vec                                                     reset_vec    000002
__Hrparam                                                        rparam       000000
__Hsfr                                                           sfr          000000
__Hsmallconst                                                    smallconst   000000
__Hspace_0                                                       (abs)        004000
__Hspace_1                                                       (abs)        00001B
__Hspace_2                                                       (abs)        000000
__Hspace_4                                                       (abs)        60000E
__Hstack                                                         stack        000000
__Hstruct                                                        struct       000000
__Htemp                                                          temp         000000
__Htext                                                          text         000000
__Htext0                                                         text0        000000
__Htext1                                                         text1        000000
__Htext10                                                        text10       000000
__Htext11                                                        text11       000000
__Htext12                                                        text12       000000
__Htext13                                                        text13       000000
__Htext14                                                        text14       000000
__Htext15                                                        text15       000000
__Htext16                                                        text16       000000
__Htext17                                                        text17       000000
__Htext18                                                        text18       000000
__Htext2                                                         text2        000000
__Htext3                                                         text3        000000
__Htext4                                                         text4        000000
__Htext5                                                         text5        000000
__Htext6                                                         text6        000000
__Htext7                                                         text7        000000
__Htext8                                                         text8        000000
__Htext9                                                         text9        000000
__LRAM                                                           (abs)        000001
__Labs1                                                          abs1         000000
__Lbank0                                                         bank0        000000
__Lbank1                                                         bank1        000000
__Lbank2                                                         bank2        000000
__Lbank3                                                         bank3        000000
__Lbank4                                                         bank4        000000
__Lbank5                                                         bank5        000000
__Lbigbss                                                        bigbss       000000
__Lbigdata                                                       bigdata      000000
__Lbigram                                                        bigram       000000
__Lbigsfr                                                        bigsfr       000000
__Lbss                                                           bss          000000
__LbssCOMRAM                                                     bssCOMRAM    000000
__Lcinit                                                         cinit        000000
__Lclrtext                                                       clrtext      000000
__Lcomram                                                        comram       000000
__Lconfig                                                        config       000000
__Lconst                                                         const        000000
__LcstackCOMRAM                                                  cstackCOMRAM 000000
__Ldata                                                          data         000000
__Leeprom_data                                                   eeprom_data  000000
__Lfarbss                                                        farbss       000000
__Lfardata                                                       fardata      000000
__Lheap                                                          heap         000000
__Libigdata                                                      ibigdata     000000
__Lidata                                                         idata        000000
__Lidloc                                                         idloc        000000
__Lifardata                                                      ifardata     000000
__Linit                                                          init         000002
__Lintcode                                                       intcode      000002
__Lintcode_body                                                  intcode_body 000000
__Lintcodelo                                                     intcodelo    000002
__Lintentry                                                      intentry     000000
__Lintret                                                        intret       000000
__Lintsave_regs                                                  intsave_regs 000000
__Lirdata                                                        irdata       000000
__Lmediumconst                                                   mediumconst  000000
__LnvCOMRAM                                                      nvCOMRAM     000000
__LnvFARRAM                                                      nvFARRAM     000000
__Lnvbit                                                         nvbit        000000
__Lnvrram                                                        nvrram       000000
__Lparam                                                         rparam       000000
__Lpowerup                                                       powerup      000002
__Lram                                                           ram          000000
__Lramtop                                                        ramtop       000600
__Lrbit                                                          rbit         000000
__Lrbss                                                          rbss         000000
__Lrdata                                                         rdata        000000
__Lreset_vec                                                     reset_vec    000000
__Lrparam                                                        rparam       000000
__Lsfr                                                           sfr          000000
__Lsmallconst                                                    smallconst   000000
__Lspace_0                                                       (abs)        000000
__Lspace_1                                                       (abs)        000000
__Lspace_2                                                       (abs)        000000
__Lspace_4                                                       (abs)        000000
__Lstack                                                         stack        000000
__Lstruct                                                        struct       000000
__Ltemp                                                          temp         000000
__Ltext                                                          text         000000
__Ltext0                                                         text0        000000
__Ltext1                                                         text1        000000
__Ltext10                                                        text10       000000
__Ltext11                                                        text11       000000
__Ltext12                                                        text12       000000
__Ltext13                                                        text13       000000
__Ltext14                                                        text14       000000
__Ltext15                                                        text15       000000
__Ltext16                                                        text16       000000
__Ltext17                                                        text17       000000
__Ltext18                                                        text18       000000
__Ltext2                                                         text2        000000
__Ltext3                                                         text3        000000
__Ltext4                                                         text4        000000
__Ltext5                                                         text5        000000
__Ltext6                                                         text6        000000
__Ltext7                                                         text7        000000
__Ltext8                                                         text8        000000
__Ltext9                                                         text9        000000
__S0                                                             (abs)        004000
__S1                                                             (abs)        00001B
__S4                                                             (abs)        000000
__S5                                                             (abs)        000000
___awdiv                                                         text10       003D44
___awdiv@counter                                                 cstackCOMRAM 00000B
___awdiv@dividend                                                cstackCOMRAM 000007
___awdiv@divisor                                                 cstackCOMRAM 000009
___awdiv@quotient                                                cstackCOMRAM 00000D
___awdiv@sign                                                    cstackCOMRAM 00000C
___awmod                                                         text9        003C68
___awmod@counter                                                 cstackCOMRAM 000005
___awmod@dividend                                                cstackCOMRAM 000001
___awmod@divisor                                                 cstackCOMRAM 000003
___awmod@sign                                                    cstackCOMRAM 000006
___heap_hi                                                       (abs)        000000
___heap_lo                                                       (abs)        000000
___inthi_sp                                                      stack        000000
___intlo_sp                                                      stack        000000
___lbdiv                                                         text16       003AA8
___lbdiv@counter                                                 cstackCOMRAM 000003
___lbdiv@dividend                                                cstackCOMRAM 000002
___lbdiv@divisor                                                 cstackCOMRAM 000001
___lbdiv@quotient                                                cstackCOMRAM 000004
___param_bank                                                    (abs)        000000
___rparam_used                                                   (abs)        000001
___sp                                                            stack        000000
___wmul                                                          text7        003A7E
___wmul@multiplicand                                             cstackCOMRAM 000003
___wmul@multiplier                                               cstackCOMRAM 000001
___wmul@product                                                  cstackCOMRAM 000005
__accesstop                                                      (abs)        000080
__activetblptr                                                   (abs)        000002
__cntErrataNOP_/tmp/xcXaGNkjc.o                                  (abs)        000001
__cntErrataNOP_dist/default/production/lab1Hector.X.production.o (abs)        000069
__end_of___awdiv                                                 text10       003E34
__end_of___awmod                                                 text9        003D44
__end_of___lbdiv                                                 text16       003B1E
__end_of___wmul                                                  text7        003AA8
__end_of__initialization                                         cinit        0039FC
__end_of_and                                                     text18       0039C4
__end_of_boot                                                    text17       003A2C
__end_of_divi                                                    text15       003A16
__end_of_main                                                    text0        004000
__end_of_nand                                                    text14       0039D2
__end_of_nor                                                     text13       0039DE
__end_of_nums                                                    text12       003A44
__end_of_or                                                      text11       0039B0
__end_of_product                                                 text8        003C68
__end_of_rest                                                    text6        003BB4
__end_of_shiftLeft                                               text5        003A5C
__end_of_shiftRight                                              text4        003A7E
__end_of_sum                                                     text3        0039F8
__end_of_xnor                                                    text2        0039EA
__end_of_xor                                                     text1        0039BA
__initialization                                                 cinit        0039F8
__mediumconst                                                    mediumconst  000000
__pbssCOMRAM                                                     bssCOMRAM    000019
__pcinit                                                         cinit        0039F8
__pcstackCOMRAM                                                  cstackCOMRAM 000001
__pnvCOMRAM                                                      nvCOMRAM     000017
__ptext0                                                         text0        003E34
__ptext1                                                         text1        0039B0
__ptext10                                                        text10       003D44
__ptext11                                                        text11       0039A6
__ptext12                                                        text12       003A2C
__ptext13                                                        text13       0039D2
__ptext14                                                        text14       0039C6
__ptext15                                                        text15       003A06
__ptext16                                                        text16       003AA8
__ptext17                                                        text17       003A16
__ptext18                                                        text18       0039BA
__ptext2                                                         text2        0039DE
__ptext3                                                         text3        0039EA
__ptext4                                                         text4        003A5C
__ptext5                                                         text5        003A44
__ptext6                                                         text6        003B1E
__ptext7                                                         text7        003A7E
__ptext8                                                         text8        003BB4
__ptext9                                                         text9        003C68
__ramtop                                                         ramtop       000600
__smallconst                                                     smallconst   000000
_and                                                             text18       0039BA
_boot                                                            text17       003A16
_divi                                                            text15       003A06
_main                                                            text0        003E34
_nand                                                            text14       0039C6
_nor                                                             text13       0039D2
_nums                                                            text12       003A2C
_or                                                              text11       0039A6
_product                                                         text8        003BB4
_rest                                                            text6        003B1E
_shiftLeft                                                       text5        003A44
_shiftRight                                                      text4        003A5C
_sum                                                             text3        0039EA
_value                                                           bssCOMRAM    000019
_xnor                                                            text2        0039DE
_xor                                                             text1        0039B0
end_of_initialization                                            cinit        0039FC
intlevel0                                                        text         0039A4
intlevel1                                                        text         0039A4
intlevel2                                                        text         0039A4
intlevel3                                                        text         0039A4
isa$std                                                          (abs)        000001
isa$xinst                                                        (abs)        000000
main@val                                                         cstackCOMRAM 000016
product@bcd                                                      cstackCOMRAM 00000F
product@d                                                        cstackCOMRAM 000010
product@mask                                                     cstackCOMRAM 000011
product@u                                                        cstackCOMRAM 000012
product@value2                                                   cstackCOMRAM 000013
rest@sig                                                         cstackCOMRAM 000007
stackhi                                                          (abs)        000000
stacklo                                                          (abs)        000000
start                                                            init         000002
start_initialization                                             cinit        0039F8
sum@temp                                                         cstackCOMRAM 000001


MODULE INFORMATION

Module		Function		Class		Link	Load	Size
/opt/microchip/xc8/v2.36/pic/sources/c99/common/lbdiv.c
		___lbdiv       		CODE           	3AA8	0000	118

/opt/microchip/xc8/v2.36/pic/sources/c99/common/lbdiv.c estimated size: 118

/opt/microchip/xc8/v2.36/pic/sources/c99/common/Umul16.c
		___wmul        		CODE           	3A7E	0000	42

/opt/microchip/xc8/v2.36/pic/sources/c99/common/Umul16.c estimated size: 42

/opt/microchip/xc8/v2.36/pic/sources/c99/common/awmod.c
		___awmod       		CODE           	3C68	0000	220

/opt/microchip/xc8/v2.36/pic/sources/c99/common/awmod.c estimated size: 220

shared
		__initialization		CODE           	39F8	0000	4

shared estimated size: 4

/opt/microchip/xc8/v2.36/pic/sources/c99/common/awdiv.c
		___awdiv       		CODE           	3D44	0000	240

/opt/microchip/xc8/v2.36/pic/sources/c99/common/awdiv.c estimated size: 240

main.c
		_product       		CODE           	3BB4	0000	180
		_shiftRight    		CODE           	3A5C	0000	34
		_boot          		CODE           	3A16	0000	22
		_xnor          		CODE           	39DE	0000	12
		_main          		CODE           	3E34	0000	460
		_nums          		CODE           	3A2C	0000	24
		_rest          		CODE           	3B1E	0000	150
		_shiftLeft     		CODE           	3A44	0000	24
		_divi          		CODE           	3A06	0000	16
		_sum           		CODE           	39EA	0000	14
		_nor           		CODE           	39D2	0000	12
		_xor           		CODE           	39B0	0000	10
		_nand          		CODE           	39C6	0000	12
		_or            		CODE           	39A6	0000	10
		_and           		CODE           	39BA	0000	10

main.c estimated size: 990

